:1000000027C218951895189518951895AAC02EC04E
:1000100018951895189518951895E199FECF109197
:10002000AE00153541F41091AF001A3A21F42EBB01
:100030000DBBE29AE19A10E01093AE0010E010932D
:10004000AF000895E199FECF34E0530F5EBBE09A14
:100050003DB33F71303009F431E04DB342954695E0
:100060004770463009F0089544E008950FB60F92A6
:1000700066E962BFA39409F4B39464E0B61611F57F
:10008000209080003090900040908100509091002E
:100090006090820070909200809083009090930016
:1000A00060916000609364006091610060936500FE
:1000B00060916200609366006091630060936700E6
:1000C000AA24BB2460916400603059F0633029F0A9
:1000D0006A2D7B2D6219730920F46BB36F606BBBC3
:1000E00003C06BB3607F6BBB000060916500603044
:1000F00059F0633029F06A2D7B2D6419750920F4BD
:100100006BB3606F6BBB03C06BB36F706BBB0000F6
:1001100060916600603059F0633029F06A2D7B2DC4
:100120006619770920F465B36F6065BB03C065B3DA
:10013000607F65BB000060916700603059F06330FC
:1001400029F06A2D7B2D6819790920F465B3606F59
:1001500065BB03C065B36F7065BB00000F900FBE39
:1001600018950FB60F923F934F930F931F936FE223
:100170006DBD60E06CBDE3946E2D633009F061C12C
:10018000EE24609180007091900080917000062FA5
:10019000172F3FEF41E0031B140B08F0880F9091DD
:1001A000680090FD25C0680F8827781F362F472FDD
:1001B0000FEF13E0301B410BB0F1009160000530F0
:1001C00089F0043079F05091A0003CDF5093A000FA
:1001D0003093700040936000009160000130E9F0BE
:1001E0000430D9F09091680091606FEF73E01BC00C
:1001F000681B8827780BBAF400916000053069F01D
:100200005091A0001FDF5093A000309370004093E6
:10021000600000916000023029F3909168009E7F99
:1002200060E070E000C0909368006093800070937D
:100230009000609181007091910080917100062F73
:10024000172F3FEF41E0031B140B08F0880F90912C
:10025000680091FD25C0680F8827781F362F472F2B
:100260000FEF13E0301B410BB0F10091610005303E
:1002700089F0043079F05091A100E4DE5093A100A0
:100280003093710040936100009161000130E9F00A
:100290000430D9F09091680092606FEF73E01BC05A
:1002A000681B8827780BBAF400916100053069F06B
:1002B0005091A100C7DE5093A1003093710040938C
:1002C000610000916100023029F3909168009D7FE8
:1002D00060E070E000C090936800609381007093CC
:1002E0009100609182007091920080917200062FBF
:1002F000172F3FEF41E0031B140B08F0880F90917C
:10030000680092FD25C0680F8827781F362F472F79
:100310000FEF13E0301B410BB0F10091620005308C
:1003200089F0043079F05091A2008CDE5093A20045
:100330003093720040936200009162000130E9F056
:100340000430D9F09091680094606FEF73E01BC0A7
:10035000681B8827780BBAF400916200053069F0B9
:100360005091A2006FDE5093A20030937200409330
:10037000620000916200023029F3909168009B7F37
:1003800060E070E000C0909368006093820070931A
:100390009200609183007091930080917300062F0A
:1003A000172F3FEF41E0031B140B08F0880F9091CB
:1003B000680093FD25C0680F8827781F362F472FC8
:1003C0000FEF13E0301B410BB0F1009163000530DB
:1003D00089F0043079F05091A30034DE5093A300EB
:1003E0003093730040936300009163000130E9F0A3
:1003F0000430D9F09091680098606FEF73E01BC0F3
:10040000681B8827780BBAF400916300053069F007
:100410005091A30017DE5093A300309373004093D4
:10042000630000916300023029F390916800977F88
:1004300060E070E000C09093680060938300709368
:1004400093001F910F914F913F910F900FBE189500
:1004500001E00EBF0FE50DBF00E00BBB08BB05BB05
:100460000FEF02BB0FEF0ABB07BB04BB02E001BBEF
:1004700005E005BF11242224332444245524662496
:10048000772488249924AA24BB24CC24DD24EE24B8
:10049000FF240027112722273327442755276627C3
:1004A000772788279927AA27BB27CC27DD27EE2780
:1004B000FF27B0E0A0E0D0E0C0E6F0E0E0E000E040
:1004C00020E009932395E9F705E50093AE000AEAD9
:1004D0000093AF00879B19C05CEFB4DD4730A9F0F3
:1004E000463099F05DEFAEDD473079F0463069F087
:1004F0005EEFA8DD473049F0463039F05FEFA2DD0E
:10050000473019F0463009F041C040E335E4A0E03F
:1005100050E0742F642F66957627872F742F632FF2
:10052000660F7627770F770F8727632F607E669594
:10053000603729F0603619F0603509F001C060E4D9
:10054000660F032F0F710C3010F00695FBCF0030B3
:1005500009F402E0062B252FA03009F4B02FA130BA
:1005600009F40B2FA13029F0889486FD0894331FDD
:10057000441FA33009F4AFEFA39585E58093AE0047
:100580008AEA8093AF0049DD539519F60CEF00938A
:10059000A0000DEF0093A1000EEF0093A2000FEF5B
:1005A0000093A300AA24BB245091A0004BDD3093FC
:1005B000700040936000409364005091A00034E0CC
:1005C000530F5093A00000916000023059F40FEFD8
:1005D0000093800003E000939000009168000E7F7C
:1005E000009368005091A1002DDD3093710040937D
:1005F0006100409365005091A10034E0530F509387
:10060000A10000916100023059F40FEF00938100C6
:1006100003E000939100009168000D7F0093680053
:100620005091A2000FDD309372004093620040931E
:1006300066005091A20034E0530F5093A200009145
:100640006200023059F40FEF0093820003E0009340
:100650009200009168000B7F009368005091A30006
:10066000F1DC309373004093630040936700509136
:10067000A30034E0530F5093A300009163000230B5
:1006800059F40FEF0093830003E00093930000916F
:100690006800077F009368002090800030909000F1
:1006A0004090810050909100609082007090920084
:1006B000809083009090930001E003BF00E002BFB0
:1006C00000E00FBD01E00EBD00E00DBD00E00CBD7F
:1006D00000E00BBD00E00ABD00E009BD00E008BD80
:1006E00000E005BD00E004BD09E109B908E10AB96F
:1006F00000E00BBF02E809BF78945F9BFECF0CB10E
:100700000635C9F411E44CD016E74AD012E748D0B8
:1007100010E246D01CE444D015E442D014E440D0AA
:1007200010E23ED011E33CD01EE23AD010E338D0C4
:1007300011E336D0E2CF023571F4F89410E01BBB20
:1007400015BB20E02EBBE09A1DB32AD02395D1F72C
:1007500010E426D07DCE073501F5F89410E01BBBE0
:1007600015BB20E05F9BFECF15E51093AE001AEAA3
:100770001093AF000CB151DC17E712D0239591F71D
:1007800010E40ED0E199FECF6DE06DBD60E06CBD70
:1007900068BF68B767FFFDCF5BCE1FE301D0ADCF69
:0A07A000312F5D9BFECF3CB9089598
:00000001FF
